:0A000000020749D2003232323232D8
:10000B00020003120055C28112005CC28002005C28
:10001B00020006C374079518FFE49400FE74802F4A
:10002B00F58274073EF583E493F4F5F8740A25180A
:10003B00F8E690075593F4F5E80518C3E51894080E
:10004B00748094804003E4F51822D28112005CD2B4
:06005B00807F0CDFFE2295
:1000630002000712073320D522AF041200A612079D
:100073003D20D517120329FF1200A6740129F9E4C4
:100083003AFA12073D20D503D51DE9020091C2813A
:0B009300120057D28102005C0200083E
:1000A300020009AE077D08EE30E704D2818002C268
:1000B30081EE25E0FE120057C28012005CDDE822CB
:1000C3000204E7AD07ED707EC28C120329FEC394D0
:1000D300037480948040037FFF22E58954FC4EF52E
:1000E30089900001120342FED394027480948040ED
:1000F300037FFF22EEFF7E007006538E7F5389FB42
:10010300EF64014E7006438E805389FBEF64024E09
:100113007003438904900002120342FFE58F54FEEB
:100123004FF58F9000031203D6E5F0F58C90000392
:100133001203D6F58A9000051203427004C28C8024
:1001430002D28C7F0022ED640160030201D6C28ECD
:10015300120329FEC394037480948040037FFF221B
:10016300EEC454F0FFE58954CF4FF5899000011296
:100173000342FED394027480948040037FFF22EEF7
:10018300FF7E007006538EBF5389BFEF64014E702C
:1001930006438E405389BFEF64024E700343894088
:1001A30090000212034225E0FFE58F54FD4FF58FC7
:1001B3009000031203D6E5F0F58D9000031203D6E9
:1001C300F58B9000051203427004C28E8002D28E1A
:1001D3007F0022ED64027061538EEF9000011203E1
:1001E30042FF7E007006538EFB538EF7EF64014E81
:1001F3007006438E04538EF7EF64024E7003438EF2
:100203000890000212034225E025E0FFE58F54FB2E
:100213004FF58F9000031203D6E5F0F5D690000357
:100223001203D6F5D7900005120342C454F0FFE53C
:100233008E54EF4FF58E7F0022ED6403706953D126
:10024300F7900001120342FED3940274809480401D
:10025300037FFF22EEFF7E00700653D1FD53D1FBD7
:10026300EF64014E700643D10253D1FBEF64024E9B
:10027300700343D104900002120342FFE5D154FE00
:100283004FF5D19000031203D6E5F0F5D4900003A7
:100293001203D6F5D590000512034233333354F8D5
:1002A300FFE5D154F78076ED6404707753D17F90E6
:1002B3000001120342FD7C00D394027480948040B9
:1002C300037FFF22ED4C700653D1DF53D1BF900063
:1002D300011203426401700643D12053D1BF900041
:1002E300011203426402700343D1409000021203DF
:1002F30042C454F0FFE5D154EF4FF5D190000312FF
:1003030003D6FDACF0ECF5D2AF058FD39000051208
:100313000342C43333335480FFE5D1547F4FF5D1C7
:100323007F00227FFF22BB010689828A83E022505D
:1003330002E722BBFE02E32289828A83E49322BB83
:10034300010CE58229F582E5833AF583E022500624
:10035300E92582F8E622BBFE06E92582F8E222E5DA
:100363008229F582E5833AF583E49322BB0106896A
:10037300828A83F0225002F722BBFE01F322BC00E3
:100383000BBE0029EF8DF084FFADF022E4CCF875AD
:10039300F008EF2FFFEE33FEEC33FCEE9DEC9840BC
:1003A30005FCEE9DFE0FD5F0E9E4CEFD22EDF8F558
:1003B300F0EE8420D21CFEADF075F008EF2FFFEDB8
:1003C30033FD4007985006D5F0F222C398FD0FD5B0
:1003D300F0EA22BB0110E58229F582E5833AF58331
:1003E300E0F5F0A3E0225009E92582F886F008E65B
:1003F30022BBFE0AE92582F8E2F5F008E222E58352
:100403002AF583E993F5F0A3E9932212071A12065A
:10041300F91206D4D2AFE4F518C201FFEFC3940872
:10042300748094805009740A2FF876100F80ED3091
:100433000114C201900000E0F50EA3E0F50FA3E064
:10044300F510A3E0F5113000E6C20012001E0517F7
:10045300E51770020516C394E8E516940340D0E44B
:10046300F516F5170509E509700205089410E50866
:1004730094274005E4F508F509AE08AF097C037D30
:10048300E81203818F12AE08AF097C037DE81203E3
:10049300817E007F64CFCDCFCECCCE1203818F136C
:1004A300AE08AF097C007D641203817E007F0ACF12
:1004B300CDCFCECCCE1203818F14AE08AF097C0012
:1004C3007D0A1203818D1585120A85130B85140C81
:1004D30085150D7B007A007912751D04E4FF120067
:1004E30066020432C0E0C083C082C0D075D000C0B1
:1004F30005C006C007AFBA43BA8090FE84E030E679
:1005030006E054BFF0807A90FE84E030E535E05495
:10051300DFF0E52260057522008066E521600D7538
:10052300210090FE87E0F5232400803490FE87E0CD
:10053300FEAD23052374002DF582E43400F583EE2C
:10054300F0803E90FE84E030E424E054EFF0E030AD
:10055300E10890FE8674FFF08027052374002523AD
:10056300F582E43400F583E090FE86F0801390FE7C
:1005730084E030E30CE054F7F0752201752101D2D9
:10058300018FBAD007D006D005D0D0D082D083D087
:10059300E03243BA80900002120342640170299052
:1005A300FE80E04440F090FE82E4F0120329543FC1
:1005B300FF90FE80E054C04FF090000312034264AA
:1005C3000190FE88702C803090FE80E054BFF09044
:1005D300FE84E4F090000412034225E0FF90FE85C0
:1005E300E054014FF0900005120342640190FE8530
:1005F3007006E054FEF08004E04401F09000011224
:10060300034290FE807006E0547FF08004E0448053
:10061300F053BA7F22EFD394017480948040037F18
:10062300FF2243BA80EF64017012ED90FE817006E1
:10063300E0547FF08011E04480F0800BEF7008906D
:10064300FE83E054874DF0EBFF7E00D39403748068
:100653009480502DEF700653B6DF53B5DFEF64017E
:100663004E700653B6DF43B520EF64024E70064367
:10067300B62053B5DFEF64034E700643B62043B58F
:10068300207F0022EFFBD39401748094805009EB08
:100693007004C2A98002D2A9EDFF7E00D394037433
:1006A3008094805029EF700553B7FDC2B9EF640100
:1006B3004E700553B7FDD2B9EF64024E700543B7D0
:1006C30002C2B9EF64034E700543B702D2B97F008B
:1006D30022E4F51B751A01751E01751D2DFB7A00A9
:1006E3007919120595E4FB7D78FF120618E5BA54D3
:1006F300CF4430F5BA22E4F519751A01F51B751CC0
:10070300A2751D40751E01FB7A007919FF1200C600
:10071300E4FD7F010206875393FC5394FC53B1F726
:1007230053B2F775CB0075CC0075E10075E200227A
:10073300AC0712000E7F5A1200A6120055A2819236
:10074300D5C28002005C787FE4F6D8FD7581230270
:10075300040E3F065B4F666D7D077F6F777C395EC6
:1007630079710040761E7038375C733E783D675070
:10077300376EBF86DBCFE6EDFD87FFEF4601020450
:05078300081020408079
:00000001FF
